:1000000008308A00AE2800000A108A100A11820700
:10001000203420342034563465347234203436345D
:100020002E3430342034203420344A3441343234B5
:1000300044345A34463400340A108A100A118207B4
:100040004134753474346F34203441346E34743434
:1000500065346E34613420346334683461346E3412
:1000600067346534723400340A108A100A1182072A
:100070004134753474346F34203441346E34743404
:1000800065346E34613420346334683461346E34E2
:1000900067346534723420347634653472343734DE
:1000A0002E3430340A3400340A108A100A118207C0
:1000B00049346634203479346F34753420347734DD
:1000C00061346E347434203474346F3420346734C3
:1000D0006F34203474346F342034653464346934BC
:1000E000743420346D346F34643465342C342034EB
:1000F000483469347434203461346E3479342034B3
:100100006B34653479340A3400340A108A100A11C9
:1001100082070A345734683465346E3420346234CC
:1001200061346E34643420346E3461346D3465343B
:1001300020342634203464346134743461342034FF
:100140007034723469346E3474342C34203459343D
:100150006F3475342034633461346E342034753434
:1001600070346434613474346534203462346134FE
:100170006E34643420346434613474346134003453
:100180000A108A100A1182074934663420346E340A
:100190006F3474342C3470346C346534613473349B
:1001A00065342034703475347334683420346534E5
:1001B0006E3474346534723420346B34653479347D
:1001C000203473346F3420346E34653478347434AE
:1001D0002034623461346E346434203464346134E5
:1001E000743461342034773469346C346C342034A2
:1001F00064346934733470346C3461347934003469
:100200000A148A100A118207713420346B34653461
:10021000793469346E342C3474346834693473340A
:10022000203472346F347534743469346E3420344D
:1002300065346E346434203461346E346434203474
:10024000683461346D346C346F34673420346D3409
:100250006F34643465342034773469346C346C34EE
:100260002034723475346E3400340A148A100A1142
:10027000820700340A148A100A11820741346E344E
:1002800074343D343E3435343434333432343134E0
:1002900000340A148A100A118207203469346E343B
:1002A00070347534743420346534723472346F347D
:1002B000723400340A148A100A11820746347234E8
:1002C000653471342E343D342034253433342E34A7
:1002D000333466344D3448347A3420342034003496
:1002E0000A148A100A1182072034773472346F346A
:1002F0007434653420340034C73084000008031996
:100300008E290630F800F701F70B8429F80B8329B2
:100310007B30F700F70B8A29800B81290034831684
:100320004608F039C700831206080F3983164704C0
:100330008312860083168610831286108316061099
:1003400083120610831606118312061583160611F2
:1003500083120611A630F700F70BAC290000003419
:10036000C730840000080319BA29B829000000002A
:10037000800BB6298A110A121E2AF03083168600D5
:1003800006108312061083168610831286148316B5
:100390000611831206150608F0398316DA000611D5
:1003A0008312061183160611831206150608F0390A
:1003B0008316DB00061183120611003083168600B7
:1003C0005B0EF7000F30F70577085A04F800831228
:1003D000003483164608C7004708F039C800831266
:1003E00006080F3983164804831286008316861088
:1003F00083128610831606108312061083160611C8
:100400008312061583160611831206118316C70E72
:10041000F030C705831206080F398316470483128C
:1004200086008316061183120615831606118312A1
:100430000611C8308316C7008312B029BD21780881
:100440008316C700C71F262A83121E2A8312003470
:100450000F308316C70083127C210030831686007C
:100460003030C60083128F2105308316C7008312F7
:100470007C2130308316C60083128F21A630F7000E
:10048000F70B402A000030308316C60083128F21FC
:1004900020308316C60083128F212E308316C600AB
:1004A0008312E92108308316C6008312E9210D303A
:1004B0008316C6008312E92106308316C600831214
:1004C000E9218A150A128D2901308316C60083128C
:1004D000E921003483165908F039DA00831206083E
:1004E0000F3983165A0483128600831686108312EE
:1004F00086108316061083120614831606118312C3
:10050000061583160611831206118316D90EF030D4
:10051000D905831206080F39831659048312860001
:10052000831606118312061583160611831206110F
:10053000BD2178088316DA00DA1FA02A8312982AD0
:10054000831200348316C6014608043C031CB62AF5
:10055000750884000008C70083120C1AB12A83169C
:10056000AC2A9900F50A8316C60AA42A83128A15B2
:100570000A12CE2AA0308316490784000008CA0058
:10058000831203178E01831603134A08831203177D
:100590008D0083168C130C1483120C08831603131E
:1005A000CB000310CB0D0310CB0D0310CB0D0310AC
:1005B000CB0DC9010318C90A490BE72A3130831250
:1005C0000C1AE42A8316DF2A9900EE2A83163030AB
:1005D00083120C1AED2A8316E82A99000310831659
:1005E000CB0DC9010318C90A490BFF2A3130831208
:1005F0000C1AFC2A8316F72A9900062B8316303032
:1006000083120C1A052B8316002B990003108316F6
:10061000CB0DC9010318C90A490B172B31308312BE
:100620000C1A142B83160F2B99001E2B83163030B7
:1006300083120C1A1D2B8316182B99000310831696
:10064000CB0DC9010318C90A490B2F2B3130831276
:100650000C1A2C2B8316272B9900362B831630303F
:1006600083120C1A352B8316302B99000310831636
:10067000CB0DC9010318C90A490B472B313083122E
:100680000C1A442B83163F2B99004E2B83163030C7
:1006900083120C1A4D2B8316482B99008316CC011C
:1006A0004C088312352100380319612B8316CC0ABC
:1006B00083120C1A5D2B8316582B99008316502B2E
:1006C00083120D300C1E622B99000A300C1E662B13
:1006D00099000034A0308316460784000008C70044
:1006E000C8013208313C031D782B0314C80C7A2B47
:1006F0000310C80C3108313C031D812B0314C80CB6
:10070000832B0310C80C3008313C031D8A2B0314C3
:10071000C80C8C2B0310C80C2F08313C031D932BE5
:100720000314C80C952B0310C80C2E08313C031D74
:100730009C2B0314C80C9E2B0310C80C0310C80C70
:100740000310C80C0310C80C831203178E01831604
:1007500003134708831203178D00831603134808F9
:10076000831203178C0083168C130C15831203134A
:100770000B08F7008B138316031755308D00AA3032
:100780008D008C148C18C22B0C1177088312031364
:100790008B048316C9014908831270218316C90A84
:1007A000F70083120C1AD62B8316D12B9900073031
:1007B00083164902031DCB2B4608C9008312BA22B7
:1007C0008A150A126D2B25122508831687008312BD
:1007D00007120830F800000000000000F817012C94
:1007E000F8138316C60C831203180716031C07128E
:1007F0007817012C7813F80BF12B00000000000093
:1008000007160130F7008401840B042CF70B032C2E
:1008100053308400840B0A2C0000F81BF02B781B4B
:10082000FA2B00340408F8000830F700A516250854
:10083000831687008312871E1F2C83161A2C83169B
:10084000C601F717352CF713352C03108312871ABE
:1008500003148316C60C7717352C7713F70B252C4A
:10086000780884004608F8004C2C013084000030E1
:10087000F71B5530F800F80B3B2C840B372C52300B
:10088000F71B1630F800F80B432C00000000F71B94
:10089000232C771B2D2C252C831200348E30F7004F
:1008A00083164708F8004608F900FA01F808031D06
:1008B000632C7908F800F9010830F702F808031DE5
:1008C000632CF7016B2C0310F81B6A2CF90DF80D43
:1008D000F703632CF81300008312003483164608D4
:1008E0000319E02CCE004A080319E02CCE07031CA4
:1008F0007A2C812C7F30CE02031CE02C0319E02CD3
:10090000852C8130CE070318E02C4E08F700F80143
:10091000F901FA014708D200D2174808D100490866
:10092000D0001830CE00CF01501CAE2C4D08FA0775
:10093000031CA02CF90A031DA02CF80A0319CF17D9
:100940004C08F907031CA72CF80A0319CF174B080A
:10095000C800C8174808F8070318CF17CF0DF80CC0
:10096000F90CFA0CD20CD10CD00C0310CE0B932C3A
:100970000130F7070318E02CF81BC52CD20DFA0D37
:10098000F90DF80DF7030319E02CD21FD62CFA0A43
:10099000031DD62CF90A031DD62CF80A031DD62CEC
:1009A000F80CF90CFA0CF70A0319E02C4708CF00F1
:1009B0004B08CF06CF1FDE2CF817E42CF813E42CDD
:1009C000F701F801F901FA010000831200348030C8
:1009D000831CED2C8316D30683128316D801D9010C
:1009E0004F08D7005308D7064E080319D92DD60053
:1009F000F70052080319E22DD60203197F2D0318C0
:100A0000022D3E2D5308DC00DC175408DB0055088E
:100A1000DA00D9010310DC0CDB0CDA0CD90CD60B94
:100A2000092DD71F162D5814F62D5810561058168C
:100A3000D13084000C2E5812D71B282D561C332D74
:100A4000DC0CDB0CDA0CD90CF70A0319F12D332D71
:100A5000DC1B362D0310D90DDA0DDB0DDC0DF70391
:100A60000319F12D282D58179E2D58134F08D70024
:100A7000CF1F3C2DDC17EA2DDC13EA2D5208D600DF
:100A8000F7004E08D6024F08DC00DC175008DB00E8
:100A90005108DA00D9010310DC0CDB0CDA0CD90C9C
:100AA000D60B4A2DD71F572DD814F62DD810561017
:100AB000D816D53084000C2ED812D71B692D561CA1
:100AC000742DDC0CDB0CDA0CD90CF70A0319F12DB0
:100AD000742DDC1B772D0310D90DDA0DDB0DDC0D29
:100AE000F7030319F12D692DD8179E2DD81353083C
:100AF000D700D31F7D2DDC17EA2DDC13EA2D530818
:100B0000DC00DC175408DB005508DA00D71F8C2DF9
:100B1000DC135815F62D5811D9015610D130840028
:100B20000C2ED71BB42D4F08D700561C9E2DDC0C65
:100B3000DB0CDA0CD90CF70A0319F12DD91FAF2DF4
:100B4000DA0A031DAF2DDB0A031DAF2DDC0A031DDE
:100B5000AF2DDC0CDB0CDA0CF70A0319F12D581B56
:100B6000352DD81B762DD32D8030DC06DC1FBC2D17
:100B7000F62D5308D700C92D4F08D700DC08031DF8
:100B8000C92DDB08031DC92DDA08031DC92DF70186
:100B9000EA2DDC1BD32D0310D90DDA0DDB0DDC0D96
:100BA000F70BC92DF12DD71FD72DDC17EA2DDC133C
:100BB000EA2D5208F7005308DC005408DB00550802
:100BC000DA00EA2D4E08F7004F08DC005008DB0081
:100BD0005108DA005C08F8005B08F9005A08FA00CE
:100BE0002B2EF701F801F901FA012B2ED901DA09B0
:100BF000DB09DC09D909D90A031D052EDA0A031D10
:100C0000052EDB0A031D052EDC0A5818152DD818F1
:100C1000562D58198B2DB92D0008DA07031C162EF6
:100C2000DB0A031D162EDC0A031956148403000880
:100C3000DB07031C1E2EDC0A03195614840300086C
:100C4000801B232E803ADC0703185614581A1B2DDC
:100C5000D81A5C2D912D00008312003483164B08A6
:100C6000D4004C08D500D601C81F382E5417D50320
:100C7000C81747080319EB2E7F304702031CA32E29
:100C8000C700D7010430D8000310CA0DC90DC80D24
:100C9000D60DD80B442E043047020318572E0330CC
:100CA0004702031DE12E0A305602031CE12E0330D9
:100CB000C702D70A8312BF2703108316CA0DC90DB6
:100CC000C80DD60D8312A52702308316D800031055
:100CD000D60CC80CC90CCA0CD80B672E8312BF27C0
:100CE00004308316D8000310CB0CCC0CCD0CCE0CEA
:100CF000D80B732E8312A527BF2783164D08CE006D
:100D00004C08CD004B08CC00CB018312A527BF2790
:100D100083164C08CE004B08CD00CB01CC018312CA
:100D2000A5278316D6194B2EC708031D9C2ECA0A69
:100D3000C90AC80AD60AE12E0310CA0DC90DC80D8A
:100D4000D60DC7034B2EC709C70A7F30C707D70187
:100D50000430D8000310CA0DC90DC80DD60DD80B2C
:100D6000AA2E0430C70705304702031CED2E83125C
:100D7000BF2703108316CA0DC90DC80DD60D031069
:100D8000CA0DC90DC80DD60D8312A52703108316F1
:100D9000CA0DC90DC80DD60DD70A0330D8000310EF
:100DA000D60CC80CC90CCA0CD80BCF2E0330C70206
:100DB000561EB32E0310D60CC80CC90CCA0CC703A0
:100DC000B32EC709C70A0330C707570AD502031C49
:100DD000D5010130EE2E0230EE2E0030D000D41BB3
:100DE000FD2ED51BFD2ED5080319FD2E2030D90070
:100DF00083126A228316D50BF62E541F042F2D3032
:100E0000D90083126A228316D41F122FD51B122FEA
:100E1000D5080319122F3030D90083126A228316A5
:100E2000D50B082FD4135413501C1D2F5708D00076
:100E30005708D200540AD207492FD01C212F540A38
:100E4000D700D4080319A32F2E30D90083126A22A9
:100E500083165708D300D30354085302031C322FC0
:100E60005408D300D30803193C2F3030D900831223
:100E70006A228316D30B352F5708D800540AD8029C
:100E80000318CB2FC703540AD2005708D2025208C6
:100E9000D0005608CF0047080319532FD100031084
:100EA000CF0CD10B4F2F52080319A32F30304F070F
:100EB000D90083126A2283165008031D672FD408B5
:100EC0000319A32F2E30D90083126A228316D00370
:100ED000D2030319A32F47080319732FD10003105E
:100EE000CF0DD10B6F2F4F08D6025608CB00480804
:100EF000CC004908CD004A08CE000310CA0DC90D28
:100F0000C80DD60D0310CA0DC90DC80DD60D4E085B
:100F1000CA07031C902FC90F902FC80F902FD60A15
:100F20004D08C907031C972FC80F972FD60A4C08E6
:100F3000C8070318D60A4B08D6070310CA0DC90DF7
:100F4000C80DD60D492F0000CB2F831283164E08F3
:100F5000CA07031CB02FC90FB02FC80FB02FD60A75
:100F60004D08C907031CB72FC80FB72FD60A4C0866
:100F7000C8070318D60A4B08D60783120034831615
:100F80005608CB004808CC004908CD004A08CE00DE
:100F9000831200348316000083128A150A128E2DE4
:100FA00083164608B63CC600FA014708CA00C717B0
:100FB0000310C70CC80CC90CFA0CF90CF80CF70C90
:100FC000C60BD82FCA1FEF2FF709F809F909FA093C
:100FD000F70A0319F80A0319F90A0319FA0A83121E
:060FE0008A150A12D02D53
:10100000F701F801F901FA018316CE01CF01D001F1
:10101000D1014D084C044B044A0403193F282030E9
:10102000D2000310C60DC70DC80DC90DCE0DCF0DD2
:10103000D00DD10D4D085102031D28284C08500237
:10104000031D28284B084F02031D28284A084E027A
:10105000031C39284A08CE024B08031C4B0FCF0251
:101060004C08031C4C0FD0024D08031C4D0FD1023D
:101070000314F70DF80DF90DFA0DD20B112800002D
:10108000CE3084008312003420308316D200CE018B
:10109000CF01D001D1014908FA004808F9004708FA
:1010A000F8004608F7000310771C64284A08CE07AA
:1010B0004B0803184B0FCF074C0803184C0FD007F1
:1010C0004D0803184D0FD107D10CD00CCF0CCE0C0E
:1010D000FA0CF90CF80CF70CD20B532883120034DD
:1010E00083164708F8014602031879284608F700D6
:1010F0008528F7010830C800C60DF70D47087702AC
:101100000318F700F80DC80B7C2883120034F70190
:10111000F8018316460803104718F707F70CF80C78
:10112000C718F707F70CF80C4719F707F70CF80C76
:10113000C719F707F70CF80C471AF707F70CF80C64
:10114000C71AF707F70CF80C471BF707F70CF80C52
:10115000C71BF707F70CF80C8312003484011F300B
:101160008305063083169F008312A0010130A10081
:10117000A201A301A401FF30A500251225088316B2
:10118000870083120716403083169900223098009A
:10119000903083129800A6013130A7002E30A800AD
:1011A0003930A9004D30AA003D30AB003330AC00DF
:1011B0002E30AD003530AE004D30AF003D30B000C8
:1011C0003430B1004D30B2002030B300B4003D30B7
:1011D000B5003730B6004D30B7002030B800B90048
:1011E0003D30BA003130BB003030BC004D30BD0066
:1011F0002030BE003D30BF003130C0003430C1006F
:101200004D30C2002030C3003D30C4003130C50035
:101210003830C6004D30C7002030C8003D30C9000E
:101220003230CA003130CB004D30CC002030CD0000
:101230003D30CE003230CF003430D0004D30D100C0
:101240002030D2003D30D3003230D4003830D500C9
:101250004D30D6002030D7003D30D8003530D90091
:101260003030DA004D30DB002030DC003D30DD0076
:101270004630DE004D30DF002030E000E1003D3040
:10128000E2003130E3003430E400E5004D30E600A8
:101290003D30E7003430E8003330E9003030EA0018
:1012A0004D30EB003D30EC00ED0103308316A00023
:1012B0000530A1000630A2000730A3000930A400C9
:1012C0000B30A5000E30A6001030A7001230A80089
:1012D0001430A9001630AA001B30AB001D30AC0042
:1012E0002930AD000A308312EE00EF00F000F1006B
:1012F0001030F200FF308316850000308600A030E9
:1013000087008312A500843083169F0083121F0874
:10131000383981389F008A11282A8A150C308316A3
:10132000C6008A118312E9218A158A1164228A155E
:101330008316C60146088A11831204208A150038D4
:101340000319AC298316C60AD9008A1183126A22AE
:101350008A1583169A298312C0308316C6008A1113
:101360008312E9218A158316C60146088A11831261
:101370001C208A1500380319C7298316C60AD9000C
:101380008A1183126A228A158316B529831283165D
:10139000C60146088A11831234208A1500380319C1
:1013A000DC298316C60A83120C1AD8298316D3297E
:1013B00099008316C92983120D300C1EDD2999006E
:1013C0000A300C1EE12999008316C60146088A11CD
:1013D000831254208A1500380319F9298316C60A86
:1013E00083120C1AF5298316F02999008316E62931
:1013F00083120D300C1EFA2999000A300C1EFE29AA
:10140000990004308316C600FA30C7008A1183128F
:101410007C218A158316C60B042AF401F30183127A
:101420008C1A272AF30A0319F40A7408C33C031C14
:10143000272A031D1F2A73084F3C031C272A10303C
:10144000F700F70B212A000083160F2A83128C1E47
:101450007B2B8316C60146088A11831285208A15C4
:10146000003803193E2A8316C60A83120C1A3A2A38
:101470008316352A990083162B2A83120D300C1EF1
:101480003F2A99000A300C1E432A99008316C60190
:1014900046088A118312C0208A15003803195B2A76
:1014A0008316C60A83120C1A572A8316522A9900E9
:1014B0008316482A83120D300C1E5C2A99000A30CC
:1014C0000C1E602A99008316C60146088A118312F1
:1014D00000218A1500380319782A8316C60A831258
:1014E0000C1A742A83166F2A99008316652A8312B0
:1014F0000D300C1E792A99000A300C1E7D2A9900A5
:1015000001308316C7008A1183127C218A158C1E34
:10151000872A1A088316B7002730F500B601360867
:101520000D3C031C712BC60146088A11831235211C
:101530008A1500380319A72A8316C60A83120C1AC3
:10154000A32A83169E2A99008316942A83120D30AB
:101550000C1EA82A99000A300C1EAC2A990083168A
:10156000C60146088A1183123A218A1500380319E8
:10157000C42A8316C60A83120C1AC02A8316BB2AF1
:1015800099008316B12A83120D300C1EC52A9900CA
:101590000A300C1EC92A99008A11A22A8A158316BC
:1015A0003608C9008A118312BA228A1505308316BB
:1015B000C600203083120C1ADF2A8316DA2A99001B
:1015C0008316C60BD92AB5013508053C031CEE2A43
:1015D000AE30350784008001B50AE42AB50135082C
:1015E000043C031C602B83128C1AF82A8316F32AFE
:1015F0001A088316B7003708713C0319602B3708A7
:101600000D3C0319602B3708303C03190B2B3708AE
:10161000313C031D1A2B370883120C1A112B831629
:101620000C2B9900AE3083163507840037088000F4
:10163000B50A5F2BC60146088A11831249218A1513
:10164000003803192E2B8316C60A83120C1A2A2B74
:101650008316252B990083161B2B83120D300C1E2D
:101660002F2B99000A300C1E332B99008316B501DD
:101670003508053C031C422BAE3035078400800141
:10168000B50A382B0530C600203083120C1A4A2BBD
:101690008316452B99008316C60B442BAE3084006D
:1016A0000030000403195E2B83120C1A592B831689
:1016B000542B00089900840A8316502BB501EF2A99
:1016C0003708713C0319712B37080D3C03196F2B38
:1016D0003608C6008A1183126A2B8A158316B60A49
:1016E0008F2A3708713C0319762B8C2A3708713CF6
:1016F00003197A2B83128A1164228A156E088316C5
:10170000C6008A118312E3238A156F088316C60068
:101710008A118312E3238A1570088316C6008A1182
:101720008312E3238A1571088316C6008A11831277
:10173000E3238A1572088316C6008A118312E323F5
:101740008A15F401F301871EB82BF30A0319F40A72
:101750007408C33C031CB82B031DB22B73084F3C09
:10176000031CB82B1030F700F70BB42B0000A32B91
:10177000871AE42B8A1112248A1578088316AE0082
:101780008A11831212248A1578088316B2008A11EE
:10179000831212248A1578088316B1008A118312E5
:1017A00012248A1578088316B0008A118312122435
:1017B0008A1578088316AF008A11831212248A15BD
:1017C00078088316B300831232308316C7008A115B
:1017D00083127C218A1583162E08B4008312031706
:1017E0008E01831603133408831203178D008316AA
:1017F0008C130C1483120C0883160313B50003100A
:10180000B50CB4010318B40AB40803190B2C8312E5
:1018100007100D2C83168312071425102508831634
:1018200087000310B50CB4010318B40AB4080319F7
:101830001D2C831287101F2C831683128714A5106A
:101840002508831687000310B50CB4010318B40AE9
:10185000B40803192F2C83120711312C831683121D
:10186000071525112508831687000310B50CB40150
:101870000318B40AB4080319412C83128711432CAE
:10188000831683128715A511250883168700031078
:10189000B50CB4010318B40AB4080319532C83120D
:1018A0008611552C83168312861583168611C7015F
:1018B0003208C6008A1183124E248A15AC30831672
:1018C000C900C530C8002730C7008330C6007A0879
:1018D000CD007908CC007808CB007708CA008A11BF
:1018E00083126E248A157A088316C5007908C4000D
:1018F0007808C3007708C200C7013108C6008A1102
:1019000083124E248A15AC308316C900C530C80036
:101910002730C7007B30C6007A08CD007908CC009C
:101920007808CB007708CA008A1183126E248A15C2
:1019300077088316C6007808C7007908C8007A08B7
:10194000C90083104908D1004808D0004708CF00DB
:101950004608CE004508D5004408D4004308D3000B
:101960004208D2008A118312E7248A157A08831666
:10197000C5007908C4007808C3007708C200C70111
:101980003008C6008A1183124E248A15AC308316A3
:10199000C900C530C8002730C7007330C6007A08B8
:1019A000CD007908CC007808CB007708CA008A11EE
:1019B00083126E248A1577088316C6007808C7003C
:1019C0007908C8007A08C90083104908D10048087E
:1019D000D0004708CF004608CE004508D50044088F
:1019E000D4004308D3004208D2008A118312E724AE
:1019F0008A157A088316C5007908C4007808C300E0
:101A00007708C200C7012F08C6008A1183124E242E
:101A10008A15AC308316C900C530C8002730C7000E
:101A20006B30C6007A08CD007908CC007808CB006E
:101A30007708CA008A1183126E248A1577088316E4
:101A4000C6007808C7007908C8007A08C900831062
:101A50004908D1004808D0004708CF004608CE000A
:101A60004508D5004408D4004308D3004208D200FA
:101A70008A118312E7248A1577088316CA0078082A
:101A8000CB007908CC007A08CD0083104D08D10036
:101A90004C08D0004B08CF004A08CE001730D500C4
:101AA000B730D4005130D3007130D2008A11831284
:101AB000E7248A157A088316C5007908C4007808D7
:101AC000C3007708C2008030C6008A118312E92162
:101AD0008A158316C60146088A1183125A218A156F
:101AE0008316C60AF700D9008A1183126A228A1562
:101AF000073083164602031D6B2D4508CA004408B3
:101B0000C9004308C8004208C700CE01CD0101301A
:101B1000CC000330CB008A1183122E2E8A150C3094
:101B20008316C70047088A1183125A218A15831623
:101B3000C70AF700D9008A1183126A228A15113068
:101B400083164702031D922D3308B4003408063C67
:101B5000031DAC2D0830B3003408073C031DB22D23
:101B60000830B3004508C9004408C8004308C7004E
:101B70004208C600CD01CC017A30CB008830CA00C3
:101B80008A1183126E248A157A088316C90079088F
:101B9000C8007808C7007708C6008A118312D02FC2
:101BA0008A157A088316BB007908BA007808B9004C
:101BB0007708B8003B08C9003A08C8003908C700D0
:101BC0003808C600CD01CC012730CB001030CA0048
:101BD0008312002077088316AF00BF01BE01BD014C
:101BE0002F08BC003F08C9003E08C8003D08C700D8
:101BF0003C08C600CD01CC012730CB001030CA0014
:101C00008312442077088316B8027808031C780FE3
:101C1000B9027908031C790FBA027A08031C7A0FFB
:101C2000BB023B08C9003A08C8003908C700380899
:101C3000C600CD01CC01CB016430CA008312002064
:101C400077088316B000BF01BE01BD013008BC009B
:101C50003F08C9003E08C8003D08C7003C08C60050
:101C6000CD01CC01CB016430CA0083124420770837
:101C700083163802B1002F08B5003508C6000A30B7
:101C8000C7008312702078088316B6003608C60095
:101C90000A30C7008312872078088316B502360EF3
:101CA000F700F030F70577083507AF003008B500CA
:101CB0003508C6000A30C7008312702078088316E2
:101CC000B6003608C6000A30C7008312872078089D
:101CD0008316B502360EF700F030F70577083507A2
:101CE000B0003108B5003508C6000A30C7008312BD
:101CF000702078088316B6003608C6000A30C70080
:101D00008312872078088316B502360EF700F0306C
:101D1000F70577083507B100B2013308B50035087B
:101D20000F39B3002F0883120C1A982E8316932EA6
:101D300099008316300883120C1AA02E83169B2E4E
:101D400099008316310883120C1AA82E8316A32E2D
:101D500099008316320883120C1AB02E8316AB2E0C
:101D600099008316330883120C1AB82E8316B32EEB
:061D700099007E2B6300C8
:02400E00723FFF
:00000001FF
